:1000000000308A00272800001030840000080319FF
:10001000182801308D008C018C0B0C288D0B0B28BF
:100020004A308C008C0B122800000000800B09283D
:10003000003411308400FC308005800C800C0008F6
:100040000319262824280000800B23287A288401FD
:100050001F308305831686148312861C6A288F013D
:100060000F08643C031C4C288316061083120614E8
:1000700083160511831205150130900004208316A4
:100080000610831206108316051183120511143011
:10009000900004208F0A30288F010F08643C031C55
:1000A000692883160610831206148316051183121D
:1000B00005150230900004208316061083120610E6
:1000C00083160511831205111430900004208F0A45
:1000D0004D282A288316061083120614831605114C
:1000E0008312051501309000042002309000EC309E
:1000F00091001928900B772883160610831206109A
:1001000083160511831205111430900004202A284B
:0201100063008A
:02400E00F93F78
:00000001FF
